:1000000000308A007D280000FF00030E8301A1005C
:100010007F08A0000A08A8008A01A00E0408A20018
:100020007708A3007808A4007908A5007A08A6003C
:100030007B08A700831383128C308400801C222845
:100040008C183528220884002308F7002408F800BB
:100050002508F9002608FA002708FB0028088A006E
:10006000210E8300FF0E7F0E09008A1147280830F9
:10007000BD02031C46283D3084000310800C00089C
:100080000319462844286400800B43280034831653
:1000900086128312861664000930BC006D30BD00E4
:1000A0003720BC0B4E282C08BB00BB0803195E2868
:1000B0006400000000000000BB0355288316861270
:1000C000831286128C108A1122283A30840000088C
:1000D00003197C280230F800BF30F7006400F70BEA
:1000E0006E28F80B6C289630F700F70B7528000087
:1000F00000006400800B6A28003484011F308305EF
:10010000703083168F001F129F121B0880399B00CE
:1001100007309C008312AB0183161F129F121B082D
:10012000803974389B001F1383121F179F17831683
:100130009F1383121F14941283160611861406123D
:100140003130831294000030831694000108C739BF
:10015000083881003030831290007830F80006387B
:1001600092008C308316920072308F000513831238
:1001700005138316851383128513831605108312C6
:1001800005108316851083128510B101B001B301EB
:10019000B2018030AC00AF0183168C14C0308312E2
:1001A0008B0483160611831206110830B900FA3049
:1001B000BA006520B90BD7282030F8001F08C739CE
:1001C00078049F000130BA0065201F151F19E6282A
:1001D0001E08F700F70CF70C3F30F7057708643E70
:1001E000AD001030F8001F08C73978049F000130B7
:1001F000BA00652020302D02B9001F151F19FE28F6
:100200001E08F700F70CF70C3F30F70577083907A1
:10021000AE000108801F0F29B11F17291129B11B3A
:100220002029B108031D17293002031C2029831639
:100230008510831285108316051083120514282952
:1002400083160510831205108316851083128510FE
:100250000108801F2E29B31F36293029B31B3F29DF
:10026000B308031D36293202031C3F298316851368
:1002700083128513831605138312051747298316E6
:1002800005138312051383168513831285136400E7
:100290000130BA0065200930B900A9018B1BA917EC
:1002A0008B136D30BD003720A91B8B17B90B4D295F
:1002B0002A08B7008316061083120610130893014C
:1002C0008316141865298312602983121308AA0063
:1002D000AA098316061083120614B501B401340866
:1002E000063C031C81292A08F7003408F80003198A
:1002F0007D290310F70CF80B79297718B50AB40A91
:100300006F293508043C0318AD29831605108312A4
:100310000510831685108312851483160513831226
:10032000051383168513831285170230B9009630A2
:10033000BA006520B90B972983160513831205139C
:1003400083168513831285138316051083120510F7
:100350008316851083128510AC29AA1FD92983160C
:1003600005138312051383168513831285178316CD
:1003700005108312051083168510831285146430CE
:10038000BA0065208316051383120513831685139F
:1003900083128513831605108312051083168510AA
:1003A000831285100430B900FA30BA006520B90B09
:1003B000D4292A1CE7295330AC00B101B001FA015D
:1003C0002E08B2007A08B3000330AB0009292A1FB7
:1003D000F529AD30AC00B301B201FA012E08B0002E
:1003E0007A08B100FD30AB000929AA1C072A673042
:1003F000AC0046302D02FA01B0007A08B100FA01D3
:100400002D08B2007A08B3000230AB000929AA1EF9
:10041000192A9930AC0046302D02FA01B2007A0850
:10042000B300FA012D08B0007A08B100FE30AB002D
:1004300009292A1D2F2A7630AC0014302D02FA012A
:10044000B0007A08B100FA012D08B2007A08B300B2
:100450000230AB002F0F2D2A2E2AAF0A09292A1E9F
:10046000452A8A30AC0014302D02FA01B2007A0815
:10047000B300FA012D08B0007A08B1000230AB00D9
:100480002F0F432A442AAF0A0929AA1D592A80306E
:10049000AC00FA012D08B0007A08B100FA012D086D
:1004A000B2007A08B300AB012F0F572A582AAF0ABF
:1004B00009292B08033C0319612A2B08FD3C031D65
:1004C000842A2F08323C0318832A831605108312CE
:1004D0000510831685108312851483160513831265
:1004E000051383168513831285174630BA006520DD
:1004F0002F08FA3C031C802A2D08AA3C0318832AE3
:0C0500003230BA006520AF010929630009
:04400E00383FFC3FFC
:00000001FF
